:020000020000FC
:100000004AC018E01A95F1F708950AE0309508946F
:1000100010F4C29A02C0C2980000F3DFF2DF3695F6
:100020000A95B1F708950AE03095089410F4DA9A29
:1000300002C0DA980000E5DFE4DF36950A95B1F7F3
:1000400008950AE03095089410F4D89A02C0D89820
:100050000000D7DFD6DF36950A95B1F7089509E09D
:10006000CF9BFECFCEDFCDDFCCDF8894CF9B089433
:100070000A9511F04795F7CF089509E0C99BFECF87
:10008000C0DFBFDFBEDF8894C99B08940A9511F0DA
:100090004795F7CF089511E01EBF1FE51DBF10E87B
:1000A00020E016BD26BDC29ABA9AD798DA9AD29A9B
:1000B000D198D89AD09A40E0D2DF342FC2DFFCCF5B
:00000001FF
